:100000000C9435000C945D000C945D000C945D0024
:100010000C945D000C945D000C945D000C945D00EC
:100020000C945D000C945D000C945D000C945D00DC
:100030000C945D000C945D000C945D000C945D00CC
:100040000C94D4010C945D000C9444020C941E0298
:100050000C945D000C945D000C945D000C945D00AC
:100060000C945D000C945D001A0311241FBECFEFA9
:10007000D8E0DEBFCDBF12E0A0E0B1E0EEE9F6E0EF
:1000800002C005900D92A83AB107D9F723E0A8EA7B
:10009000B2E001C01D92AE34B207E1F710E0C5E353
:1000A000D0E004C02197FE010E944703C433D1076A
:1000B000C9F70E9476020C944D030C9400003FB7E0
:1000C000F8948091AD029091AE02A091AF02B091F0
:1000D000B00226B5A89B05C02F3F19F00196A11DBF
:1000E000B11D3FBFBA2FA92F982F8827BC01CD0182
:1000F000620F711D811D911D42E0660F771F881FE1
:10010000991F4A95D1F708958F929F92AF92BF920F
:10011000CF92DF92EF92FF920E945F004B015C0151
:1001200088EBC82E8BE0D82EE12CF12C0E945F00CA
:10013000681979098A099B09683E73408105910510
:10014000A8F321E0C21AD108E108F10888EE880E70
:1001500083E0981EA11CB11CC114D104E104F10478
:1001600029F7FF90EF90DF90CF90BF90AF909F90D6
:100170008F900895AF92BF92CF92DF92EF92FF924D
:100180000F931F93CF93DF936C017B018B01040FBF
:10019000151FEB015E01AE18BF08C017D10759F05B
:1001A0006991D601ED91FC910190F081E02DC6019D
:1001B0000995892B79F7C501DF91CF911F910F9197
:1001C000FF90EF90DF90CF90BF90AF900895FC012B
:1001D000538D448D252F30E0842F90E0821B930BAC
:1001E000541710F0CF96089501970895FC01918D52
:1001F000828D981761F0A28DAE0FBF2FB11D5D9655
:100200008C91928D9F5F9F73928F90E008958FEFF6
:100210009FEF0895FC01918D828D981731F0828DAA
:10022000E80FF11D858D90E008958FEF9FEF089501
:10023000FC01918D228D892F90E0805C9F4F821B65
:1002400091098F739927089581EB92E00E9418011C
:1002500021E0892B09F420E0822F089580E090E0CE
:10026000892B29F00E94240181110C94000008952B
:10027000FC01A48DA80FB92FB11DA35ABF4F2C911B
:10028000848D90E001968F739927848FA689B78912
:100290002C93A089B1898C91837080648C93938D09
:1002A000848D981306C00288F389E02D80818F7DAC
:1002B00080830895EF92FF920F931F93CF93DF9364
:1002C000EC0181E0888F9B8D8C8D98131AC0E88992
:1002D000F989808185FF15C09FB7F894EE89FF8961
:1002E0006083E889F98980818370806480839FBFFF
:1002F00081E090E0DF91CF911F910F91FF90EF90FF
:100300000895F62E0B8D10E00F5F1F4F0F7311270E
:10031000E02E8C8D8E110CC00FB607FCFACFE88949
:10032000F989808185FFF5CFCE010E943801F1CF98
:10033000EB8DEC0FFD2FF11DE35AFF4FF0829FB7BD
:10034000F8940B8FEA89FB8980818062CFCFCF93AD
:10035000DF93EC01888D8823B9F0AA89BB89E889ED
:10036000F9898C9185FD03C0808186FD0DC00FB693
:1003700007FCF7CF8C9185FFF2CF808185FFEDCF11
:10038000CE010E943801E9CFDF91CF910895FC01A1
:1003900001900020E9F73197AF01481B590BBC01D0
:1003A00081EB92E00C94BA001F920F920FB60F925D
:1003B00011242F933F938F939F93AF93BF9380917B
:1003C000A9029091AA02A091AB02B091AC02309127
:1003D000A80223E0230F2D3758F50196A11DB11D6A
:1003E0002093A8028093A9029093AA02A093AB0243
:1003F000B093AC028091AD029091AE02A091AF0299
:10040000B091B0020196A11DB11D8093AD029093F1
:10041000AE02A093AF02B093B002BF91AF919F9193
:100420008F913F912F910F900FBE0F901F901895B5
:1004300026E8230F0296A11DB11DD2CF1F920F9265
:100440000FB60F9211242F933F934F935F936F93A7
:100450007F938F939F93AF93BF93EF93FF9381EB22
:1004600092E00E943801FF91EF91BF91AF919F916F
:100470008F917F916F915F914F913F912F910F904D
:100480000FBE0F901F9018951F920F920FB60F92EC
:1004900011242F938F939F93EF93FF93E091C102C9
:1004A000F091C2028081E091C702F091C80282FD02
:1004B0001BC090818091CA028F5F8F732091CB0205
:1004C000821741F0E091CA02F0E0EF54FD4F958FA2
:1004D0008093CA02FF91EF919F918F912F910F907E
:1004E0000FBE0F901F9018958081F4CF789484B53B
:1004F000826084BD84B5816084BD85B5826085BD20
:1005000085B5816085BD80916E00816080936E00AD
:10051000109281008091810082608093810080919F
:100520008100816080938100809180008160809350
:1005300080008091B10084608093B1008091B00010
:1005400081608093B00080917A00846080937A000B
:1005500080917A00826080937A0080917A00816035
:1005600080937A0080917A00806880937A0010925C
:10057000C100E091C102F091C20282E08083E0916B
:10058000BD02F091BE021082E091BF02F091C00264
:100590008FEC80831092C902E091C502F091C602EF
:1005A00086E08083E091C302F091C4028081806183
:1005B0008083E091C302F091C402808188608083CF
:1005C000E091C302F091C402808180688083E09151
:1005D000C302F091C40280818F7D8083C2E400E079
:1005E00010E0C0937C0080917A00806480937A0050
:1005F00080917A0086FDFCCF8091780090917900FF
:10060000883E9340A4F482E191E00E94C7018DE20C
:1006100091E00E94C7010E9484000115110509F3B1
:100620000E9424018823E9F20E940000DACF80E3CF
:1006300091E0EBCFE1EBF2E01382128288EE93E0DF
:10064000A0E0B0E084839583A683B78384E091E043
:100650009183808385EC90E09587848784EC90E09B
:100660009787868780EC90E0918B808B81EC90E07F
:10067000938B828B82EC90E0958B848B86EC90E060
:10068000978B868B118E128E138E148E0895EE0F1B
:0E069000FF1F0590F491E02D0994F894FFCF20
:10069E00000000005A01BA00E700A7011801F60099
:1006AE000A016E656564203556206F6E20416E61BD
:1006BE006C6F67696320706F72742032000D0A00D0
:1006CE003738203131312031313920333220313237
:1006DE003120313131203131372033322031303732
:1006EE002031313020313131203131392033322037
:1006FE003635203131302039372031303820313104
:10070E003120313033203130352039392033322009
:10071E0031313220313035203131302031313520F8
:10072E0033322039392039372031313020333220DD
:10073E0039372031313520313037203332203130C6
:10074E0032203131312031313420333220313132C7
:10075E0020313131203131392031303120313134B5
:10076E0020313020313136203130342031303120BB
:10077E003332203130322031303820393720313089
:10078E003320333220313032203131312031313487
:10079E002033322033392037382031313120333273
:1007AE002031313220313131203131392031303167
:1007BE00203131342033322031313020313131206B
:1007CE003332203130322031303820393720313039
:1007DE00332033392033322031303520313135203A
:1007EE003332203538203332203637203834203714
:1007FE003020343520363820373620383320313209
:10080E0033203533203836203935203131362034F7
:10081E0038203935203834203130342035312039E4
:10082E0035203737203131312034382031313020E6
:08083E00333320313235000094
:00000001FF
